:020000040000FA
:04080000D8EF06F037
:1008100003B20AEF05F0F2B425EF05F09EB02DEF1C
:1008200005F09EB235EF05F0F2A81AEF04F0F2B22F
:100830001CEF04F087EF06F0CD90F2929EA026EF19
:1008400004F00101533F26EF04F0542BAEC1B2F186
:10085000AFC1B3F1B0C1B4F1B1C1B5F1AAC1AEF14C
:10086000ABC1AFF1ACC1B0F1ADC1B1F1A6C1AAF15C
:10087000A7C1ABF1A8C1ACF1A9C1ADF1A2C1A6F16C
:10088000A3C1A7F1A4C1A8F1A5C1A9F19EC1A2F17C
:100890009FC1A3F1A0C1A4F1A1C1A5F19AC19EF18C
:1008A0009BC19FF19CC1A0F19DC1A1F196C19AF19C
:1008B00097C19BF198C19CF199C19DF1CECF96F162
:1008C000CFCF97F153C198F154C199F1CF6ACE6A55
:1008D0000101536B546B9E90CD800FBC0F8E0FBAED
:1008E00075EF04F00F8A87EF06F00F8C0FBEB1EFA3
:1008F00004F096C19AF197C19BF198C19CF199C1FE
:100900009DF19AC19EF19BC19FF19CC1A0F19DC137
:10091000A1F19EC1A2F19FC1A3F1A0C1A4F1A1C107
:10092000A5F1A2C1A6F1A3C1A7F1A4C1A8F1A5C1D7
:10093000A9F1A6C1AAF1A7C1ABF1A8C1ACF1A9C1A7
:10094000ADF1AAC1AEF1ABC1AFF1ACC1B0F1ADC177
:10095000B1F1AEC1B2F1AFC1B3F1B0C1B4F1B1C147
:10096000B5F101015E6B5F6B606B616B96515E2749
:1009700097515F2398516023995161239A515E27C3
:100980009B515F239C5160239D5161239E515E27A3
:100990009F515F23A0516023A1516123A2515E2783
:1009A000A3515F23A4516023A5516123A6515E2763
:1009B000A7515F23A8516023A9516123AA515E2743
:1009C000AB515F23AC516023AD516123AE515E2723
:1009D000AF515F23B0516023B1516123B2515E2703
:1009E000B3515F23B4516023B5516123D890010105
:1009F000613360335F335E33D8900101613360331C
:100A00005F335E33D8900101613360335F335E330F
:100A100087EF06F00392030103EE00F080517F0B95
:100A2000E92604C0EFFF802B8151805D700BD8A4B4
:100A30008B8200008051815D700BD8A48B92815114
:100A40008019D8B4079087EF06F0F2940101453F72
:100A500087EF06F0462B87EF06F09E900101533F8B
:100A600087EF06F0542B87EF06F09E92C3CF55F127
:100A7000C4CF56F1C28207B4A0EF05F047C14BF1D5
:100A800048C14CF149C14DF14AC14EF15EC162F11C
:100A90005FC163F160C164F161C165F196C1B6F1F6
:100AA00097C1B7F198C1B8F199C1B9F19AC1BAF13A
:100AB0009BC1BBF19CC1BCF19DC1BDF19EC1BEF10A
:100AC0009FC1BFF1A0C1C0F1A1C1C1F1A2C1C2F1DA
:100AD000A3C1C3F1A4C1C4F1A5C1C5F1A6C1C6F1AA
:100AE000A7C1C7F1A8C1C8F1A9C1C9F1AAC1CAF17A
:100AF000ABC1CBF1ACC1CCF1ADC1CDF1AEC1CEF14A
:100B0000AFC1CFF1B0C1D0F1B1C1D1F1B2C1D2F119
:100B1000B3C1D3F1B4C1D4F1B5C1D5F1010155517F
:100B20005B2756515C23E86A5D230E2EA0EF05F08B
:100B30005CC157F15DC158F15B6B5C6B5D6B078EFF
:100B40000201002F87EF06F03C0E006F00C10CF190
:100B500001C10DF102C10EF103C10FF104C110F189
:100B600005C111F106C112F107C113F108C114F159
:100B700009C115F10AC116F10BC117F134C135F1E4
:100B800001018A67CBEF05F08B67CBEF05F08C672F
:100B9000CBEF05F08D67CFEF05F0FFEF05F08EC1CD
:100BA00000F18FC101F190C102F191C103F1010186
:100BB000010E046F000E056F000E066F000E076F2A
:100BC000A7EC14F000C18EF101C18FF102C190F1C8
:100BD00003C191F10067F4EF05F00167F4EF05F050
:100BE0000267F4EF05F00367FFEF05F08AC18EF1AD
:100BF0008BC18FF18CC190F18DC191F10F80D57EA9
:100C0000D5BE69D0D6CF47F1D7CF48F145C149F11C
:100C1000E86AE8CF4AF1109047C100F148C101F1FC
:100C200049C102F14AC103F101010A0E046F000E2D
:100C3000056F000E066F000E076FA7EC14F003AFF0
:100C40001080010154A731EF06F00F9A0F9C0F9E00
:100C50000101000E5E6F600E5F6F3D0E606F080E4B
:100C6000616F010147BF41EF06F0486741EF06F0B1
:100C7000496741EF06F04A6741EF06F0F28866EFF8
:100C800006F0F2985E6B5F6B606B616B966B976BB7
:100C9000986B996B9A6B9B6B9C6B9D6B9E6B9F6B20
:100CA000A06BA16BA26BA36BA46BA56BA66BA76BD0
:100CB000A86BA96BAA6BAB6BAC6BAD6BAE6BAF6B80
:100CC000B06BB16BB26BB36BB46BB56BD76AD66AF2
:100CD0000101456B466B0CC100F10DC101F10EC164
:100CE00002F10FC103F110C104F111C105F112C1EC
:100CF00006F113C107F114C108F115C109F116C1BC
:100D00000AF117C10BF135C134F187EF06F002C0CB
:100D1000E0FF005001C0D8FF1000A6B28DEF06F032
:100D20000CC0A9FF0BC0A8FFA69EA69CA684F29E9D
:100D3000550EA76EAA0EA76EA682F28EA694A6B234
:100D40009FEF06F00C2A1200A96EA69EA69CA68014
:100D5000A8500C2A120004012C0E826F61EC08F0DE
:100D6000A2EC15F00C50A4EC06F0E8CF00F10C500A
:100D7000A4EC06F0E8CF01F101AFC4EF06F00101E9
:100D8000FF0E026FFF0E036F45EC15F02967D0EFE1
:100D900006F00401200E826F61EC08F0D5EF06F03A
:100DA00004012D0E826F61EC08F06FEC13F012005D
:100DB000076A0F6A106A0F010E0EC16E860EC06EB2
:100DC000030EC26E0F01896A110E926E080E8A6EB2
:100DD000F10E936E8B6A800E946EF18E0E6A010195
:100DE0005B6B5C6B5D6B576B586BF29A0101476BE9
:100DF000486B496B4A6B4B6B4C6B4D6B4E6B4F6B3F
:100E0000506B516B526B456B466BD76AD66A0F01BC
:100E1000280ED56EF28A9D90B00ECD6E01015E6BEC
:100E20005F6B606B616B626B636B646B656B666B56
:100E3000676B686B696B536B546BCF6ACE6A0F9AA2
:100E40000F9C0F9E9D80760ECA6E9D8202013C0E05
:100E5000006FCC6A160EA4EC06F0E8CF00F1170E76
:100E6000A4EC06F0E8CF01F1180EA4EC06F0E8CFF0
:100E700002F1190EA4EC06F0E8CF03F1010103AF73
:100E80005CEF07F0A2EC15F0160E0C6E00C10BF033
:100E90008DEC06F0170E0C6E01C10BF08DEC06F018
:100EA000180E0C6E02C10BF08DEC06F0190E0C6ED4
:100EB00003C10BF08DEC06F000C18AF101C18BF18A
:100EC00002C18CF103C18DF100C18EF101C18FF11E
:100ED00002C190F103C191F11A0EA4EC06F0E8CF23
:100EE00000F11B0EA4EC06F0E8CF01F11C0EA4ECFF
:100EF00006F0E8CF02F11D0EA4EC06F0E8CF03F1F6
:100F0000010103AFB2EF07F0A2EC15F01A0E0C6E60
:100F100000C10BF08DEC06F01B0E0C6E01C10BF046
:100F20008DEC06F01C0E0C6E02C10BF08DEC06F081
:100F30001D0E0C6E03C10BF08DEC06F01A0EA4EC26
:100F400006F0E8CF00F11B0EA4EC06F0E8CF01F1AB
:100F50001C0EA4EC06F0E8CF02F11D0EA4EC06F086
:100F6000E8CF03F100C192F101C193F102C194F104
:100F700003C195F1240EAC6E900EAB6E240EAC6ED8
:100F8000080EB86E000EB06E1F0EAF6E0401806BBF
:100F9000816B0F01900EAB6E0F019D8A0301806B78
:100FA000816BC26B8B9207900001F28EF28C07B0BE
:100FB0001CEF12F00FB0FDEF0CF00301805181190E
:100FC0007F0BD8B41CEF12F013EE00F081517F0BB1
:100FD000E126812BE7CFE8FFE00BD8B41CEF12F03D
:100FE00023EE82F0C2513F0BD926E7CFDFFFC22BA1
:100FF000DF50780AD8A41CEF12F007808EC100F1F0
:101000008FC101F190C102F191C103F10101040E00
:10101000046F000E056F000E066F000E076FA7EC41
:1010200014F000AF1DEF08F00101030E8E6F000EEB
:101030008F6F000E906F000E916F03018251720A44
:10104000D8B4FDEF0CF08251520AD8B4FDEF0CF089
:101050008251750AD8B4FDEF0CF08251630AD8B4FE
:10106000D8EF0EF08251690AD8B4B8EF09F0825176
:101070007A0AD8B4CBEF0AF08251490AD8B457EFB4
:1010800009F08251500AD8B475EF08F08251700A05
:10109000D8B4B8EF08F08251540AD8B4E3EF08F09E
:1010A0008251740AD8B429EF09F08251730AD8B476
:1010B0002DEF0CF08251530AD8B492EF0CF00DEFE3
:1010C0000FF0040114EE00F080517F0BE12682C482
:1010D000E7FF802B120004010D0E826F61EC08F017
:1010E0000A0E826F61EC08F0120083C32AF184C3F8
:1010F0002BF185C32CF186C32DF187C32EF188C354
:101100002FF189C330F18AC331F18BC332F18CC323
:1011100033F10101F0EC15F067EC15F0160E0C6ED2
:1011200000C10BF08DEC06F0170E0C6E01C10BF038
:101130008DEC06F0180E0C6E02C10BF08DEC06F073
:10114000190E0C6E03C10BF08DEC06F000C18AF194
:1011500001C18BF102C18CF103C18DF100C18EF18F
:1011600001C18FF102C190F103C191F157EF09F074
:1011700083C32AF184C32BF185C32CF186C32DF1DF
:1011800087C32EF188C32FF189C330F18AC331F1AF
:101190008BC332F18CC333F10101F0EC15F067EC35
:1011A00015F000C18AF101C18BF102C18CF103C1BC
:1011B0008DF100C18EF101C18FF102C190F103C127
:1011C00091F157EF09F083C32AF184C32BF185C352
:1011D0002CF186C32DF187C32EF188C32FF189C36B
:1011E00030F18AC331F18CC332F18DC333F1010187
:1011F000F0EC15F067EC15F00101000E046F000E25
:10120000056F010E066F000E076FB8EC14F01A0E92
:101210000C6E00C10BF08DEC06F01B0E0C6E01C1C4
:101220000BF08DEC06F01C0E0C6E02C10BF08DEC79
:1012300006F01D0E0C6E03C10BF08DEC06F000C124
:1012400092F101C193F102C194F103C195F157EFFD
:1012500009F083C32AF184C32BF185C32CF186C323
:101260002DF187C32EF188C32FF189C330F18AC3D2
:1012700031F18CC332F18DC333F10101F0EC15F083
:1012800067EC15F00101000E046F000E056F010EF2
:10129000066F000E076FB8EC14F000C192F101C1A7
:1012A00093F102C194F103C195F157EF09F0160EC5
:1012B000A4EC06F0E8CF00F1170EA4EC06F0E8CF9E
:1012C00001F1180EA4EC06F0E8CF02F1190EA4EC1F
:1012D00006F0E8CF03F145EC15F028EC13F004011B
:1012E000730E826F61EC08F004012C0E826F61ECCA
:1012F00008F08AC100F18BC101F18CC102F18DC1EE
:1013000003F145EC15F028EC13F00401730E826F25
:1013100061EC08F004012C0E826F61EC08F01A0EEB
:10132000A4EC06F0E8CF00F11B0EA4EC06F0E8CF29
:1013300001F11C0EA4EC06F0E8CF02F11D0EA4ECA6
:1013400006F0E8CF03F128EC0FF004012C0E826FB9
:1013500061EC08F092C100F193C101F194C102F176
:1013600095C103F128EC0FF06BEC08F00DEF0FF0D6
:101370000401690E826F61EC08F004012C0E826F8B
:1013800061EC08F00101040E006F000E016F000E09
:10139000026F000E036F45EC15F02CC182F40401BE
:1013A000300E822761EC08F02DC182F40401300E6A
:1013B000822761EC08F02EC182F40401300E8227EE
:1013C00061EC08F02FC182F40401300E822761EC39
:1013D00008F030C182F40401300E822761EC08F07D
:1013E00031C182F40401300E822761EC08F032C171
:1013F00082F40401300E822761EC08F033C182F4DC
:101400000401300E822761EC08F004012C0E826F7B
:1014100061EC08F00101030E006F000E016F000E79
:10142000026F000E036F45EC15F02CC182F404012D
:10143000300E822761EC08F02DC182F40401300ED9
:10144000822761EC08F02EC182F40401300E82275D
:1014500061EC08F02FC182F40401300E822761ECA8
:1014600008F030C182F40401300E822761EC08F0EC
:1014700031C182F40401300E822761EC08F032C1E0
:1014800082F40401300E822761EC08F033C182F44B
:101490000401300E822761EC08F004012C0E826FEB
:1014A00061EC08F00101200E006F000E016F000ECC
:1014B000026F000E036F45EC15F02CC182F404019D
:1014C000300E822761EC08F02DC182F40401300E49
:1014D000822761EC08F02EC182F40401300E8227CD
:1014E00061EC08F02FC182F40401300E822761EC18
:1014F00008F030C182F40401300E822761EC08F05C
:1015000031C182F40401300E822761EC08F032C14F
:1015100082F40401300E822761EC08F033C182F4BA
:101520000401300E822761EC08F004012C0E826F5A
:1015300061EC08F0200EF86EF76AF66A0401090003
:10154000F5CF82F461EC08F00900F5CF82F461EC8C
:1015500008F00900F5CF82F461EC08F00900F5CF3E
:1015600082F461EC08F00900F5CF82F461EC08F038
:101570000900F5CF82F461EC08F00900F5CF82F4A0
:1015800061EC08F00900F5CF82F461EC08F06BEC37
:1015900008F00DEF0FF08351630AD8A40DEF0FF0A0
:1015A0008451610AD8A40DEF0FF085516C0AD8A4BC
:1015B0000DEF0FF08651410A42E08651440A1BE0CC
:1015C0008651420AD8B432EF0BF08651350AD8B4AE
:1015D00097EF10F08651360AD8B4ECEF10F0865130
:1015E000370AD8B455EF11F08651380AD8B4B3EFA2
:1015F00011F00DEF0FF00798079A04017A0E826F31
:1016000061EC08F00401780E826F61EC08F00401CF
:10161000640E826F61EC08F081A816EF0BF00401F4
:10162000550E826F61EC08F01BEF0BF004014C0EBD
:10163000826F61EC08F06BEC08F00DEF0FF007889B
:10164000079A04017A0E826F61EC08F00401410EE2
:10165000826F61EC08F00401610E826F61EC08F0AA
:101660000CEF0BF00798078A04017A0E826F61EC89
:1016700008F00401420E826F61EC08F00401610E73
:10168000826F61EC08F00CEF0BF00101666750EF20
:101690000BF0676750EF0BF0686750EF0BF069676E
:1016A00068EF0BF04F675CEF0BF050675CEF0BF0EF
:1016B00051675CEF0BF0526768EF0BF00101000E11
:1016C000006F000E016F000E026F000E036F12001C
:1016D0000101620E046F010E056F000E066F000E11
:1016E000076F66C100F167C101F168C102F169C10C
:1016F00003F1A7EC14F003BFECEF0BF00101000EB7
:10170000046FA80E056F550E066F020E076F66C1B7
:1017100000F167C101F168C102F169C103F166C15D
:1017200086F167C187F168C188F169C189F1A7ECC9
:1017300014F003BFA5EF0BF00101000E866FA80E99
:10174000876F550E886F020E896F0E0EA4EC06F09F
:10175000E8CF18F10F0EA4EC06F0E8CF19F1100E47
:10176000A4EC06F0E8CF1AF1110EA4EC06F0E8CFD5
:101770001BF1F0EC13F086C104F187C105F188C1BB
:1017800006F189C107F1A7EC14F00782B4EC13F05D
:10179000F0EC13F00792B4EC13F086C100F187C1AE
:1017A00001F188C102F189C103F10792B4EC13F091
:1017B000CC0E046FE00E056F870E066F050E076FE7
:1017C000A7EC14F000C118F101C119F102C11AF11E
:1017D00003C11BF124EF0CF00101800E006F1A0E03
:1017E000016F060E026F000E036F4FC104F150C16E
:1017F00005F151C106F152C107F1A7EC14F003AF96
:1018000005EF0CF0A2EC15F012000E0EA4EC06F0A1
:10181000E8CF18F10F0EA4EC06F0E8CF19F1100E86
:10182000A4EC06F0E8CF1AF1110EA4EC06F0E8CF14
:101830001BF14FC100F150C101F151C102F152C180
:1018400003F10782B4EC13F018C100F119C101F1E2
:101850001AC102F11BC103F112000401730E826F61
:1018600061EC08F004012C0E826F61EC08F0078433
:1018700062C166F163C167F164C168F165C169F174
:101880004BC14FF14CC150F14DC151F14EC152F11C
:1018900057C159F158C15AF1079453EC0CF06BEC55
:1018A00008F00DEF0FF066C100F167C101F168C1EA
:1018B00002F169C103F1010145EC15F028EC13F0C8
:1018C0000401630E826F61EC08F004012C0E826F3C
:1018D00061EC08F04FC100F150C101F151C102F1BA
:1018E00052C103F1010145EC15F028EC13F004019D
:1018F000660E826F61EC08F004012C0E826F61ECC1
:1019000008F0A2EC15F059C100F15AC101F1010132
:1019100045EC15F028EC13F00401740E826F61ECB5
:1019200008F0120010820401530E826F61EC08F07F
:1019300004012C0E826F61EC08F083C32AF184C38A
:101940002BF185C32CF186C32DF187C32EF188C3FB
:101950002FF189C330F18AC331F18BC332F18CC3CB
:1019600033F10101F0EC15F067EC15F000C166F100
:1019700001C167F102C168F103C169F18EC32AF1A7
:101980008FC32BF190C32CF191C32DF192C32EF193
:1019900093C32FF194C330F195C331F196C332F163
:1019A00097C333F10101F0EC15F067EC15F000C1BD
:1019B0004FF101C150F102C151F103C152F1E3EC09
:1019C00015F099C32FF19AC330F19BC331F19CC339
:1019D00032F19DC333F10101F0EC15F067EC15F025
:1019E00000C159F101C15AF153EC0CF004012C0E65
:1019F000826F61EC08F004EF0DF08251520A03E1AE
:101A00000F8204EF0DF00F928251750A03E11084EA
:101A10000BEF0DF010948251550A03E1108612EF7E
:101A20000DF01096078410B26FEF0DF010A45BEF6D
:101A30000DF0B6C166F1B7C167F1B8C168F1B9C1BF
:101A400069F1BAC16AF1BBC16BF1BCC16CF1BDC136
:101A50006DF1BEC16EF1BFC16FF1C0C170F1C1C106
:101A600071F1C2C172F1C3C173F1C4C174F1C5C1D6
:101A700075F1C6C176F1C7C177F1C8C178F1C9C1A6
:101A800079F1CAC17AF1CBC17BF1CCC17CF1CDC176
:101A90007DF1CEC17EF1CFC17FF1D0C180F1D1C146
:101AA00081F1D2C182F1D3C183F1D4C184F1D5C116
:101AB00085F163EF0DF062C166F163C167F164C146
:101AC00068F165C169F14BC14FF14CC150F14DC195
:101AD00051F14EC152F157C159F158C15AF1079411
:101AE0000FA091EF0DF0010192677EEF0DF093676B
:101AF0007EEF0DF094677EEF0DF0956782EF0DF0AD
:101B000091EF0DF045EC0BF092C104F193C105F19A
:101B100094C106F195C107F1A7EC14F003BFD5EF0E
:101B20000EF045EC0BF00101000E046F000E056F86
:101B3000010E066F000E076FD8EC14F010A4A8EF8A
:101B40000DF00401750E826F61EC08F0ADEF0DF041
:101B50000401720E826F61EC08F004012C0E826F9A
:101B600061EC08F045EC15F02967BCEF0DF00401BD
:101B7000200E826FBFEF0DF004012D0E826F61EC1D
:101B800008F030C182F40401300E822761EC08F0C5
:101B900031C182F40401300E822761EC08F00401A7
:101BA0002E0E826F61EC08F032C182F40401300E17
:101BB000822761EC08F033C182F40401300E8227E1
:101BC00061EC08F004016D0E826F61EC08F0040115
:101BD0002C0E826F61EC08F04FC100F150C101F191
:101BE00051C102F152C103F1010145EC15F028EC9D
:101BF00013F00401480E826F61EC08F004017A0EC4
:101C0000826F61EC08F004012C0E826F61EC08F029
:101C100066C100F167C101F168C102F169C103F158
:101C2000010145EC15F028EC13F00401630E826FFE
:101C300061EC08F004012C0E826F61EC08F066C1C3
:101C400000F167C101F168C102F169C103F101014D
:101C50000A0E046F000E056F000E066F000E076F70
:101C6000B8EC14F0000E046F120E056F000E066F34
:101C7000000E076FD8EC14F045EC15F02AC182F481
:101C80000401300E822761EC08F02BC182F40401BC
:101C9000300E822761EC08F02CC182F40401300E72
:101CA000822761EC08F02DC182F40401300E8227F6
:101CB00061EC08F02EC182F40401300E822761EC41
:101CC00008F02FC182F40401300E822761EC08F085
:101CD00030C182F40401300E822761EC08F0040167
:101CE0002E0E826F61EC08F031C182F40401300ED7
:101CF000822761EC08F032C182F40401300E8227A1
:101D000061EC08F033C182F40401300E822761ECEB
:101D100008F00401730E826F61EC08F004012C0ED0
:101D2000826F61EC08F0A2EC15F059C100F15AC1C4
:101D300001F137EC10F00FB2A1EF0EF00FA0D3EFCE
:101D40000EF004012C0E826F61EC08F0200EF86E8C
:101D5000F76AF66A04010900F5CF82F461EC08F035
:101D60000900F5CF82F461EC08F00900F5CF82F4A8
:101D700061EC08F00900F5CF82F461EC08F009008D
:101D8000F5CF82F461EC08F00900F5CF82F461EC44
:101D900008F00900F5CF82F461EC08F00900F5CFF6
:101DA00082F461EC08F06BEC08F00F900DEF0FF08F
:101DB0000401630E826F61EC08F004012C0E826F47
:101DC00061EC08F013EC0FF004012C0E826F61EC53
:101DD00008F086EC0FF004012C0E826F61EC08F025
:101DE00002EC10F004012C0E826F61EC08F001018E
:101DF000F80E006FCD0E016F660E026F030E036FBB
:101E000028EC0FF004012C0E826F61EC08F018EC46
:101E100010F06BEC08F00DEF0FF00301C26B0790B0
:101E200010921CEF12F0D8900E0EA4EC06F0E8CF42
:101E300000F10F0EA4EC06F0E8CF01F1100EA4ECB7
:101E400006F0E8CF02F1110EA4EC06F0E8CF03F1A2
:101E50000101000E046F000E056F010E066F000EEB
:101E6000076FD8EC14F045EC15F02AC182F4040198
:101E7000300E822761EC08F02BC182F40401300E91
:101E8000822761EC08F02CC182F40401300E822715
:101E900061EC08F02DC182F40401300E822761EC60
:101EA00008F02EC182F40401300E822761EC08F0A4
:101EB0002FC182F40401300E822761EC08F030C19A
:101EC00082F40401300E822761EC08F031C182F403
:101ED0000401300E822761EC08F004012E0E826F9F
:101EE00061EC08F032C182F40401300E822761EC0B
:101EF00008F033C182F40401300E822761EC08F04F
:101F000004016D0E826F61EC08F01200120EA4EC59
:101F100006F0E8CF00F1130EA4EC06F0E8CF01F1D3
:101F2000140EA4EC06F0E8CF02F1150EA4EC06F0B6
:101F3000E8CF03F101010A0E046F000E056F000ED9
:101F4000066F000E076FB8EC14F0000E046F120E4F
:101F5000056F000E066F000E076FD8EC14F045EC0D
:101F600015F02AC182F40401300E822761EC08F0DA
:101F70002BC182F40401300E822761EC08F02CC1E1
:101F800082F40401300E822761EC08F02DC182F446
:101F90000401300E822761EC08F02EC182F40401A6
:101FA000300E822761EC08F02FC182F40401300E5C
:101FB000822761EC08F030C182F40401300E8227E0
:101FC00061EC08F004012E0E826F61EC08F031C163
:101FD00082F40401300E822761EC08F032C182F4F1
:101FE0000401300E822761EC08F033C182F4040151
:101FF000300E822761EC08F00401730E826F61ECF1
:1020000008F012000A0EA4EC06F0E8CF00F10B0E67
:10201000A4EC06F0E8CF01F10C0EA4EC06F0E8CF3A
:1020200002F10D0EA4EC06F0E8CF03F137EF10F04B
:10203000060EA4EC06F0E8CF00F1070EA4EC06F0C3
:10204000E8CF01F1080EA4EC06F0E8CF02F1090E8A
:10205000A4EC06F0E8CF03F137EF10F00101A2EC99
:1020600015F0078457C100F158C101F1079401012F
:10207000E80E046F800E056F000E066F000E076FEE
:10208000B8EC14F0000E046F040E056F000E066F1E
:10209000000E076FD8EC14F0880E046F130E056F56
:1020A000000E066F000E076FA7EC14F00A0E046F07
:1020B000000E056F000E066F000E076FD8EC14F0CF
:1020C00045EC15F0010129676BEF10F00401200EBB
:1020D000826F6EEF10F004012D0E826F61EC08F03C
:1020E00030C182F40401300E822761EC08F031C166
:1020F00082F40401300E822761EC08F032C182F4D0
:102100000401300E822761EC08F004012E0E826F6C
:1021100061EC08F033C182F40401300E822761ECD7
:1021200008F00401430E826F61EC08F0120087C3CF
:102130002AF188C32BF189C32CF18AC32DF18BC3FB
:102140002EF18CC32FF18DC330F18EC331F190C3CA
:1021500032F191C333F10101296BF0EC15F067EC1A
:1021600015F00101000E046F000E056F010E066FE1
:10217000000E076FB8EC14F00E0E0C6E00C10BF0E1
:102180008DEC06F00F0E0C6E01C10BF08DEC06F01D
:10219000100E0C6E02C10BF08DEC06F0110E0C6EE1
:1021A00003C10BF08DEC06F004017A0E826F61EC36
:1021B00008F004012C0E826F61EC08F00401350E6A
:1021C000826F61EC08F004012C0E826F61EC08F064
:1021D00013EC0FF01BEF0BF087C32AF188C32BF130
:1021E00089C32CF18AC32DF18BC32EF18CC32FF13F
:1021F0008DC330F18EC331F190C332F191C333F10D
:102200000101296BF0EC15F067EC15F0880E046FF6
:10221000130E056F000E066F000E076FACEC14F086
:10222000000E046F040E056F000E066F000E076FA0
:10223000B8EC14F00101E80E046F800E056F000E7B
:10224000066F000E076FD8EC14F00A0E0C6E00C17A
:102250000BF08DEC06F00B0E0C6E01C10BF08DEC4B
:1022600006F00C0E0C6E02C10BF08DEC06F00D0E9C
:102270000C6E03C10BF08DEC06F004017A0E826F38
:1022800061EC08F004012C0E826F61EC08F004018F
:10229000360E826F61EC08F004012C0E826F61EC47
:1022A00008F002EC10F01BEF0BF087C32AF188C393
:1022B0002BF189C32CF18AC32DF18BC32EF18CC372
:1022C0002FF18DC330F18FC331F190C332F191C33F
:1022D00033F10101F0EC15F067EC15F0000E046F1E
:1022E000120E056F000E066F000E076FB8EC14F0AB
:1022F00001010A0E046F000E056F000E066F000E3E
:10230000076FD8EC14F0120E0C6E00C10BF08DECC0
:1023100006F0130E0C6E01C10BF08DEC06F0140EDE
:102320000C6E02C10BF08DEC06F0150E0C6E03C1A5
:102330000BF08DEC06F004017A0E826F61EC08F070
:1023400004012C0E826F61EC08F00401370E826FDD
:1023500061EC08F004012C0E826F61EC08F086EC51
:102360000FF01BEF0BF087C32AF188C32BF189C351
:102370002CF18AC32DF18BC32EF18CC32FF18DC3A9
:1023800030F18EC331F190C332F191C333F10101C9
:10239000296BF0EC15F067EC15F0880E046F130E46
:1023A000056F000E066F000E076FACEC14F0000E08
:1023B000046F040E056F000E066F000E076FB8EC79
:1023C00014F00101E80E046F800E056F000E066F19
:1023D000000E076FD8EC14F0060E0C6E00C10BF067
:1023E0008DEC06F0070E0C6E01C10BF08DEC06F0C3
:1023F000080E0C6E02C10BF08DEC06F0090E0C6E8F
:1024000003C10BF08DEC06F004017A0E826F61ECD3
:1024100008F004012C0E826F61EC08F00401380E04
:10242000826F61EC08F004012C0E826F61EC08F001
:1024300018EC10F01BEF0BF081A8DAEF12F007A8F0
:1024400093EF12F00101800E006F1A0E016F060E5D
:10245000026F000E036F4BC104F14CC105F14DC179
:1024600006F14EC107F1A7EC14F003BFDAEF12F04A
:1024700022EC13F04BC100F14CC101F14DC102F14E
:102480004EC103F10782B4EC13F018C104F119C175
:1024900005F11AC106F11BC107F1F80E006FCD0E50
:1024A000016F660E026F030E036FA7EC14F00E0EA1
:1024B0000C6E00C10BF08DEC06F00F0E0C6E01C11E
:1024C0000BF08DEC06F0100E0C6E02C10BF08DECD3
:1024D00006F0110E0C6E03C10BF08DEC06F00784B4
:1024E0000101A2EC15F057C100F158C101F10794A8
:1024F0000A0E0C6E00C10BF08DEC06F00B0E0C6E8C
:1025000001C10BF08DEC06F00C0E0C6E02C10BF04D
:102510008DEC06F00D0E0C6E03C10BF08DEC06F089
:102520000798DAEF12F007AADAEF12F00784010138
:10253000A2EC15F057C100F158C101F10794060E45
:102540000C6E00C10BF08DEC06F0070E0C6E01C195
:102550000BF08DEC06F0080E0C6E02C10BF08DEC4A
:1025600006F0090E0C6E03C10BF08DEC06F007842B
:1025700062C100F163C101F164C102F165C103F1FF
:102580000794120E0C6E00C10BF08DEC06F0130ECA
:102590000C6E01C10BF08DEC06F0140E0C6E02C136
:1025A0000BF08DEC06F0150E0C6E03C10BF08DECEC
:1025B00006F0079A0401805181197F0B0BE09EA859
:1025C00009D014EE00F081517F0BE126E750812BFA
:1025D0000F01AD6ED7EF07F018C100F119C101F17D
:1025E0001AC102F11BC103F1000E046F000E056F4A
:1025F000010E066F000E076FD8EC14F029A117EF3B
:1026000013F02051D8B417EF13F018C100F119C11D
:1026100001F11AC102F11BC103F1000E046F000E9B
:10262000056F0A0E066F000E076FD8EC14F012004B
:102630000101045100130551011306510213075102
:10264000031312000101186B196B1A6B1B6B12003C
:102650002AC182F40401300E822761EC08F02BC1FC
:1026600082F40401300E822761EC08F02CC182F460
:102670000401300E822761EC08F02DC182F40401C0
:10268000300E822761EC08F02EC182F40401300E76
:10269000822761EC08F02FC182F40401300E8227FA
:1026A00061EC08F030C182F40401300E822761EC45
:1026B00008F031C182F40401300E822761EC08F089
:1026C00032C182F40401300E822761EC08F033C17C
:1026D00082F40401300E822761EC08F012002FC151
:1026E00082F40401300E822761EC08F030C182F4DC
:1026F0000401300E822761EC08F031C182F404013C
:10270000300E822761EC08F032C182F40401300EF1
:10271000822761EC08F033C182F40401300E822775
:1027200061EC08F01200060E116E060E126E060E17
:10273000136E112E99EF13F0122E99EF13F0132E42
:1027400099EF13F08B84020E116E020E126E020EC0
:10275000136E112EA9EF13F0122EA9EF13F0132E02
:10276000A9EF13F08B9412000101005305E101530E
:1027700003E1025301E1002B77EC14F0A2EC15F019
:102780003951006F3A51016F420E046F4B0E056FC5
:10279000000E066F000E076FB8EC14F000C104F1D4
:1027A00001C105F102C106F103C107F118C100F131
:1027B00019C101F11AC102F11BC103F107B2E5EF22
:1027C00013F0ACEC14F0E7EF13F0A7EC14F000C139
:1027D00018F101C119F102C11AF103C11BF1120074
:1027E000A2EC15F059C100F15AC101F1060EA4EC9A
:1027F00006F0E8CF04F1070EA4EC06F0E8CF05F1EF
:10280000080EA4EC06F0E8CF06F1090EA4EC06F0E1
:10281000E8CF07F1A7EC14F000C124F101C125F1C4
:1028200002C126F103C127F1290E046F000E056FC6
:10283000000E066F000E076FB8EC14F0EE0E046F7A
:10284000430E056F000E066F000E076FACEC14F020
:1028500024C104F125C105F126C106F127C107F104
:10286000B8EC14F000C11CF101C11DF102C11EF150
:1028700003C11FF1120EA4EC06F0E8CF04F1130E11
:10288000A4EC06F0E8CF05F1140EA4EC06F0E8CFB6
:1028900006F1150EA4EC06F0E8CF07F10D0E006F5F
:1028A000000E016F000E026F000E036FB8EC14F003
:1028B000180E046F000E056F000E066F000E076FF6
:1028C000D8EC14F01CC104F11DC105F11EC106F1C4
:1028D0001FC107F1ACEC14F06A0E046F2A0E056FED
:1028E000000E066F000E076FA7EC14F01200BF0E6B
:1028F000FA6E200E3A6F396BD890003701370237E5
:102900000337D8B088EF14F03A2F7DEF14F0390771
:102910003A070353D8B412000331070B80093F6F05
:1029200003390F0B010F396F80EC5FF0406F3905F1
:1029300080EC5FF0405D405F396B3F33D8B03927A2
:1029400039333FA99DEF14F040513927120001019E
:10295000C7EC15F0D8B01200010103510719346F0C
:102960008AEC15F0D8900751031934AF800F12008C
:102970000101346BAEEC15F0D8A0C4EC15F0D8B062
:10298000120099EC15F0A2EC15F01F0E366FDAEC80
:1029900015F00B35D8B08AEC15F0D8A00335D8B0B7
:1029A0001200362FC7EF14F034B1B1EC15F012005D
:1029B0000101346B04510511061107110008D8A05C
:1029C000AEEC15F0D8A0C4EC15F0D8B01200086B2E
:1029D000096B0A6B0B6BDAEC15F01F0E366FDAEC35
:1029E00015F007510B5DD8A402EF15F006510A5DF2
:1029F000D8A402EF15F00551095DD8A402EF15F037
:102A00000451085DD8A015EF15F00451085F055179
:102A1000D8A0053D095F0651D8A0063D0A5F0751C1
:102A2000D8A0073D0B5FD8900081362FEFEF14F050
:102A300034B1B1EC15F0346BAEEC15F0D890DEEC9F
:102A400015F007510B5DD8A432EF15F006510A5D61
:102A5000D8A432EF15F00551095DD8A432EF15F076
:102A60000451085DD8A041EF15F0003F41EF15F08B
:102A7000013F41EF15F0023F41EF15F0032BD8B4B1
:102A8000120034B1B1EC15F012000101346BAEEC60
:102A900015F0D8B01200E3EC15F0200E366F0037B9
:102AA00001370237033711EE33F00A0E376FE7367E
:102AB0000A0EE75CD8B0E76EE552372F57EF15F0F6
:102AC000362F4FEF15F034B12981D8901200010153
:102AD0000A0E346F200E366F11EE29F03451376F25
:102AE0000A0ED890E652D8B0E726E732372F72EFB9
:102AF00015F00333023301330033362F6CEF15F03A
:102B0000E750FF0FD8A00335D8B0120029B1B1ECBF
:102B100015F01200045100270551D8B0053D0127DA
:102B20000651D8B0063D02270751D8B0073D03270C
:102B300012000051086F0151096F02510A6F0351D1
:102B40000B6F12000101006B016B026B036B120033
:102B50000101046B056B066B076B12000335D8A0EF
:102B600012000351800B001F011F021F031F003FB3
:102B7000C1EF15F0013FC1EF15F0023FC1EF15F0B5
:102B8000032B342B032512000735D8A01200075160
:102B9000800B041F051F061F071F043FD7EF15F00A
:102BA000053FD7EF15F0063FD7EF15F0072B342B75
:102BB0000725120000370137023703370837093776
:102BC0000A370B3712000101296B2A6B2B6B2C6B18
:102BD0002D6B2E6B2F6B306B316B326B336B1200A6
:102BE00001012A510F0B2A6F2B510F0B2B6F2C5108
:102BF0000F0B2C6F2D510F0B2D6F2E510F0B2E6FB6
:102C00002F510F0B2F6F30510F0B306F31510F0BB6
:102C1000316F32510F0B326F33510F0B336F120084
:10BF0000E844F926000C160C2B0C3F0C520C640C68
:10BF1000760C860C960CA50CB30CC10CCF0CDC0C6B
:06BF2000E80CF40C000C1B
:00000001FF
